:1000000002195F75E11543E12022320221BA121C68
:100010002512164B0200FE5397DE3202220075C5F0
:10002000602222021E2AE4F5AC75C830439A404390
:10003000C9107598D075CBFF75CAF49002F574FCA1
:10004000F0A37490F0D2CA43B81043B71043A8107D
:0A005000D2B322021EE043E11022A9
:06005B000200170220E084
:10006300021E859002E3EBF0A3EAF0A3E9F0E4FEBD
:100073009002E3E0FBA3E0FAA3E0F98E827583002C
:10008300120FD325E0FDEFA806088002C313D8FCA6
:1000930054014D8E827583001210120EEEB408D0F7
:1000A300E4FE9002E3E0FBA3E0FAA3E0F98E82759D
:1000B3008300120FD35407FF70179002E6E0FBA3EF
:1000C300E0FAA3E0F9120FBAFFEE902AC4935F801F
:1000D30019EFB407189002E6E0FBA3E0FAA3E0F9F6
:1000E300120FBAFFEE902ACC934F1210000EEEB40B
:0600F30008B02202137F99
:1000FB0002000A9002DC7401F0A37400F0A3740EEA
:10010B00F0A37401F0A37400F0A37422F07B017AC6
:10011B0002790F12208D9002DC7401F0A37400F0B1
:10012B00A37436F0A37401F0A37400F0A3744AF027
:10013B007B017A02791712208D9002DC7401F0A3F7
:10014B007400F0A3745EF0A37401F0A37400F0A329
:10015B007472F07B017A02791F12208D9002DC748D
:10016B0001F0A37400F0A37486F0A37401F0A374E0
:10017B0000F0A3749AF07B017A02792712208D90FC
:10018B00005DE0FF900049E04FFF900035E0FE90EE
:10019B000021E04E4FFF900085E0FE900071E04E95
:1001AB004FFF9000ADE0FE900099E04E4FF52920F7
:1001BB00650302066A204A0302066A900052E0FCBD
:1001CB00A3E0FDA3E0FEA3E0FF90003EE0F8A3E078
:1001DB00F9A3E0FAA3E04FFFEA4EFEE94DFDE84C30
:1001EB00FCC004C005C006AB0790002AE0FCA3E0EE
:1001FB00FDA3E0FEA3E0FF900016E0F8A3E0F9A357
:10020B00E0FAA3E04FFFEA4EFEE94DFDE84CFCD0CF
:10021B0002D001D000EF4BFFEE4AFEED49FDEC485A
:10022B00FCC004C005C006AB0790007AE0FCA3E05D
:10023B00FDA3E0FEA3E0FF900066E0F8A3E0F9A3C6
:10024B00E0FAA3E04FFFEA4EFEE94DFDE84CFCD08F
:10025B0002D001D000EB4FFFEA4EFEE94DFDE84C1A
:10026B00FCC004C005C006AB079000A2E0FCA3E0F5
:10027B00FDA3E0FEA3E0FF90008EE0F8A3E0F9A35E
:10028B00E0FAA3E04FFFEA4EFEE94DFDE84CFCD04F
:10029B0002D001D000EB4FF50BEA4EF50AE94DF514
:1002AB0009E84CF508900056E0FCA3E0FDA3E0FE46
:1002BB00A3E0FF900042E0F8A3E0F9A3E0FAA3E08B
:1002CB004FFFEA4EFEE94DFDE84CFCC004C005C0F3
:1002DB0006AB0790002EE0FCA3E0FDA3E0FEA3E03D
:1002EB00FF90001AE0F8A3E0F9A3E0FAA3E04FFFB8
:1002FB00EA4EFEE94DFDE84CFCD002D001D000EFF8
:10030B004BFFEE4AFEED49FDEC48FCC004C005C0B6
:10031B0006AB0790007EE0FCA3E0FDA3E0FEA3E0AC
:10032B00FF90006AE0F8A3E0F9A3E0FAA3E04FFF27
:10033B00EA4EFEE94DFDE84CFCD002D001D000EBBB
:10034B004FFFEA4EFEE94DFDE84CFCC004C005C072
:10035B0006AB079000A6E0FCA3E0FDA3E0FEA3E044
:10036B00FF900092E0F8A3E0F9A3E0FAA3E04FFFBF
:10037B00EA4EFEE94DFDE84CFCD002D001D000EB7B
:10038B004FF50FEA4EF50EE94DF50DE84CF50C7BEC
:10039B00017A0279377D081224BE7B017A02793FFC
:1003AB007D081224BE7B017A0279477D081224BE98
:1003BB007B017A02794F7D081224BE7B007A00798B
:1003CB0008122246EF70030205F43048030204E8DA
:1003DB00900022E0FCA3E0FDA3E0FEA3E0FF900071
:1003EB000EE0F8A3E0F9A3E0FAA3E04FFFEA4EFE1C
:1003FB00E94DFDE84CFCEF550BF513EE550AF512E4
:10040B00ED5509F511EC5508F510900026E0FCA30D
:10041B00E0FDA3E0FEA3E0FF900012E0F8A3E0F9FB
:10042B00A3E0FAA3E04FFFEA4EFEE94DFDE84CFCDA
:10043B00EF550FF517EE550EF516ED550DF515ECB1
:10044B00550CF5149002F2E4F0A37400F0A37410B1
:10045B00F07B017A0279371222CE90004AE0FCA39E
:10046B00E0FDA3E0FEA3E0FF900036E0F8A3E0F987
:10047B00A3E0FAA3E04FFFEA4EFEE94DFDE84CFC8A
:10048B00EF550BF513EE550AF512ED5509F511EC79
:10049B005508F51090004EE0FCA3E0FDA3E0FEA391
:1004AB00E0FF90003AE0F8A3E0F9A3E0FAA3E04FF5
:1004BB00FFEA4EFEE94DFDE84CFCEF550FF517EE4C
:1004CB00550EF516ED550DF515EC550CF514900272
:1004DB00F2E4F0A37400F0A3741002063E900072D5
:1004EB00E0FCA3E0FDA3E0FEA3E0FF90005EE0F8DC
:1004FB00A3E0F9A3E0FAA3E04FFFEA4EFEE94DFDBE
:10050B00E84CFCEF550BF513EE550AF512ED5509BA
:10051B00F511EC5508F510900076E0FCA3E0FDA377
:10052B00E0FEA3E0FF900062E0F8A3E0F9A3E0FA9D
:10053B00A3E04FFFEA4EFEE94DFDE84CFCEF550FF3
:10054B00F517EE550EF516ED550DF515EC550CF59D
:10055B00149002F2E4F0A37400F0A37410F07B018A
:10056B007A0279471222CE90009AE0FCA3E0FDA319
:10057B00E0FEA3E0FF900086E0F8A3E0F9A3E0FA29
:10058B00A3E04FFFEA4EFEE94DFDE84CFCEF550BA7
:10059B00F513EE550AF512ED5509F511EC5508F565
:1005AB001090009EE0FCA3E0FDA3E0FEA3E0FF9013
:1005BB00008AE0F8A3E0F9A3E0FAA3E04FFFEA4ECC
:1005CB00FEE94DFDE84CFCEF550FF517EE550EF51A
:1005DB0016ED550DF515EC550CF5149002F2E4F0F3
:1005EB00A37400F0A37410806C2049192048169056
:1005FB0002F2E4F0A37400F0A37408F07B017A021A
:10060B007937020C842049193048169002F2E4F035
:10061B00A37400F0A37408F07B017A027947020CF3
:10062B00843049192048169002F2E4F0A37400F0CC
:10063B00A37408F07B017A02793F020C84204903F2
:10064B00020C87204803020C879002F2E4F0A3749B
:10065B0000F0A37408F07B017A02794F020C8490AE
:10066B00002AE0FCA3E0FDA3E0FEA3E0FF90001650
:10067B00E0F8A3E0F9A3E0FAA3E04FF50BEA4EF59F
:10068B000AE94DF509E84CF50890002EE0FCA3E0D3
:10069B00FDA3E0FEA3E0FF90001AE0F8A3E0F9A3AE
:1006AB00E0FAA3E04FF50FEA4EF50EE94DF50DE834
:1006BB004CF50C900052E0FCA3E0FDA3E0FEA3E0A0
:1006CB00FF90003EE0F8A3E0F9A3E0FAA3E04FF5BA
:1006DB0013EA4EF512E94DF511E84CF51090005662
:1006EB00E0FCA3E0FDA3E0FEA3E0FF900042E0F8F6
:1006FB00A3E0F9A3E0FAA3E04FF517EA4EF516E9EC
:10070B004DF515E84CF5147B007A0079081222465A
:10071B00EF700302082E900022E0FCA3E0FDA3E0A3
:10072B00FEA3E0FF90000EE0F8A3E0F9A3E0FAA32C
:10073B00E04FFFEA4EFEE94DFDE84CFCEF550BF5A3
:10074B001BEE550AF51AED5509F519EC5508F51878
:10075B00900026E0FCA3E0FDA3E0FEA3E0FF9000E9
:10076B0012E0F8A3E0F9A3E0FAA3E04FFFEA4EFE94
:10077B00E94DFDE84CFCEF550FF51FEE550EF51E40
:10078B00ED550DF51DEC550CF51C9002F2E4F0A3A4
:10079B007400F0A37418F07B017A0279371222CE21
:1007AB0090004AE0FCA3E0FDA3E0FEA3E0FF900075
:1007BB0036E0F8A3E0F9A3E0FAA3E04FFFEA4EFE20
:1007CB00E94DFDE84CFCEF550BF51BEE550AF51A00
:1007DB00ED5509F519EC5508F51890004EE0FCA302
:1007EB00E0FDA3E0FEA3E0FF90003AE0F8A3E0F900
:1007FB00A3E0FAA3E04FFFEA4EFEE94DFDE84CFC07
:10080B00EF550FF51FEE550EF51EED550DF51DECC5
:10081B00550CF51C9002F2E4F0A37400F0A37418CD
:10082B0002096B7B007A007910122246EF700302EB
:10083B000949900022E0FCA3E0FDA3E0FEA3E0FF4A
:10084B0090000EE0F8A3E0F9A3E0FAA3E04FFFEA73
:10085B004EFEE94DFDE84CFCEF5513F51BEE551222
:10086B00F51AED5511F519EC5510F518900026E019
:10087B00FCA3E0FDA3E0FEA3E0FF900012E0F8A3D1
:10088B00E0F9A3E0FAA3E04FFFEA4EFEE94DFDE8E5
:10089B004CFCEF5517F51FEE5516F51EED5515F5DE
:1008AB001DEC5514F51C9002F2E4F0A37400F0A3B8
:1008BB007418F07B017A0279371222CE90004AE04D
:1008CB00FCA3E0FDA3E0FEA3E0FF900036E0F8A35D
:1008DB00E0F9A3E0FAA3E04FFFEA4EFEE94DFDE895
:1008EB004CFCEF5513F51BEE5512F51AED5511F5A2
:1008FB0019EC5510F51890004EE0FCA3E0FDA3E0B9
:10090B00FEA3E0FF90003AE0F8A3E0F9A3E0FAA31E
:10091B00E04FFFEA4EFEE94DFDE84CFCEF5517F5B5
:10092B001FEE5516F51EED5515F51DEC5514F51C62
:10093B009002F2E4F0A37400F0A3741880229002EA
:10094B00F2E4F0A37400F0A37408F07B017A02794F
:10095B00371222CE9002F2E4F0A37400F0A37410CD
:10096B00F07B017A02793F1222CE90007AE0FCA351
:10097B00E0FDA3E0FEA3E0FF900066E0F8A3E0F942
:10098B00A3E0FAA3E04FF50BEA4EF50AE94DF509A2
:10099B00E84CF50890007EE0FCA3E0FDA3E0FEA38D
:1009AB00E0FF90006AE0F8A3E0F9A3E0FAA3E04FC0
:1009BB00F50FEA4EF50EE94DF50DE84CF50C9000F0
:1009CB00A2E0FCA3E0FDA3E0FEA3E0FF90008EE01D
:1009DB00F8A3E0F9A3E0FAA3E04FF513EA4EF51202
:1009EB00E94DF511E84CF5109000A6E0FCA3E0FDF5
:1009FB00A3E0FEA3E0FF900092E0F8A3E0F9A3E0F0
:100A0B00FAA3E04FF517EA4EF516E94DF515E84C4C
:100A1B00F5147B007A007908122246EF7003020B63
:100A2B0040900072E0FCA3E0FDA3E0FEA3E0FF908A
:100A3B00005EE0F8A3E0F9A3E0FAA3E04FFFEA4E73
:100A4B00FEE94DFDE84CFCEF550BF51BEE550AF599
:100A5B001AED5509F519EC5508F518900076E0FCE0
:100A6B00A3E0FDA3E0FEA3E0FF900062E0F8A3E0AB
:100A7B00F9A3E0FAA3E04FFFEA4EFEE94DFDE84C87
:100A8B00FCEF550FF51FEE550EF51EED550DF51D33
:100A9B00EC550CF51C9002F2E4F0A37400F0A37477
:100AAB0018F07B017A0279471222CE90009AE0FC73
:100ABB00A3E0FDA3E0FEA3E0FF900086E0F8A3E037
:100ACB00F9A3E0FAA3E04FFFEA4EFEE94DFDE84C37
:100ADB00FCEF550BF51BEE550AF51AED5509F519FB
:100AEB00EC5508F51890009EE0FCA3E0FDA3E0FE9A
:100AFB00A3E0FF90008AE0F8A3E0F9A3E0FAA3E0FB
:100B0B004FFFEA4EFEE94DFDE84CFCEF550FF51F8C
:100B1B00EE550EF51EED550DF51DEC550CF51C9017
:100B2B0002F2E4F0A37400F0A37418F07B017A02D4
:100B3B00794F020C847B007A007910122246EF70F9
:100B4B0003020C5B900072E0FCA3E0FDA3E0FEA3AC
:100B5B00E0FF90005EE0F8A3E0F9A3E0FAA3E04F1A
:100B6B00FFEA4EFEE94DFDE84CFCEF5513F51BEE8D
:100B7B005512F51AED5511F519EC5510F5189000A5
:100B8B0076E0FCA3E0FDA3E0FEA3E0FF900062E0B3
:100B9B00F8A3E0F9A3E0FAA3E04FFFEA4EFEE94D1C
:100BAB00FDE84CFCEF5517F51FEE5516F51EED55F0
:100BBB0015F51DEC5514F51C9002F2E4F0A374002E
:100BCB00F0A37418F07B017A0279471222CE9000C1
:100BDB009AE0FCA3E0FDA3E0FEA3E0FF900086E01B
:100BEB00F8A3E0F9A3E0FAA3E04FFFEA4EFEE94DCC
:100BFB00FDE84CFCEF5513F51BEE5512F51AED55B0
:100C0B0011F519EC5510F51890009EE0FCA3E0FDD2
:100C1B00A3E0FEA3E0FF90008AE0F8A3E0F9A3E0D5
:100C2B00FAA3E04FFFEA4EFEE94DFDE84CFCEF5511
:100C3B0017F51FEE5516F51EED5515F51DEC551454
:100C4B00F51C9002F2E4F0A37400F0A37418802258
:100C5B009002F2E4F0A37400F0A37408F07B017A25
:100C6B000279471222CE9002F2E4F0A37400F0A3B3
:100C7B007410F07B017A02794F1222CE2290030D71
:100C8B00EFF0900258E0540FFE25E0247BF582E450
:100C9B00342AF583E493FDEF75F013A424AEF582AB
:100CAB00E43400F583EDF0EE25E0247CF582E434AA
:100CBB002AF583E493FEEF75F013A424AFF582E4D9
:100CCB003400F583EEF0E4F529900257E0F528A205
:100CDB0040924CA241924DA242924EA244924F534B
:100CEB0029F0EF75F013A424AFF582E43400F583FB
:100CFB00E04529F0900259E0FEEF75F013A424B003
:100D0B00F582E43400F583EEF090025AE0FEEF75C5
:100D1B00F013A424B1F582E43400F583EEF0EF7503
:100D2B00F013A424B2F582E43400F583E4F09002CE
:100D3B0081E0FEEF75F013A424B3F582E43400F5E3
:100D4B0083EEF0900282E0FEEF75F013A424B4F56D
:100D5B0082E43400F583EEF0900283E0FEEF75F051
:100D6B0013A424B5F582E43400F583EEF0EF75F0AF
:100D7B0013A424BEF582E43400F583E0F529EF14C7
:100D8B00602F14604814606C147003020E26240448
:100D9B006003020E399002EC7401F0A37402F0A30D
:100DAB007461F07B017A0079B612238E90025D801C
:100DBB00369002EC7401F0A37402F0A37469F07B1B
:100DCB00017A0079C912238E90025D80419002EC6A
:100DDB007401F0A37402F0A37471F07B017A0079B3
:100DEB00DC12238E90025EE0F528A2419248A242CB
:100DFB009249803A9002EC7401F0A37402F0A37450
:100E0B0079F07B017A0079EF12238E90025EE0F588
:100E1B0028A2449248A2459249801378027C017D16
:100E2B00017B017A02798A7E007F08120F9490026F
:100E3B005CE0F528A245924AA246924BA247924CFF
:100E4B00A243924D900258E0F528A246924E900391
:100E5B000DE0FF75F013A424BEF582E43400F58396
:100E6B00E529F0300003121566900284E04440FF40
:100E7B0090030DE0FE75F013A424BFF582E434005B
:100E8B00F583EFF0900285E0FFEE75F013A424C01C
:100E9B00F582E43400F583EFF090025FE0F529A2D0
:100EAB004D924F532980EE75F013A424BFF582E4C5
:100EBB003400F583E04529F022E709F608DFFA80D4
:100ECB0046E709F208DFFA803E88828C83E709F057
:100EDB00A3DFFA8032E309F608DFFA8078E309F240
:100EEB0008DFFA807088828C83E309F0A3DFFA8035
:100EFB006489828A83E0A3F608DFFA805889828AA4
:100F0B0083E0A3F208DFFA804C80D280FA80C6809F
:100F1B00D4806980F28033801080A680EA809A802A
:100F2B00A880DA80E280CA803389828A83ECFAE473
:100F3B0093A3C8C582C8CCC583CCF0A3C8C582C84F
:100F4B00CCC583CCDFE9DEE7800D89828A83E4930D
:100F5B00A3F608DFF9ECFAA9F0EDFB2289828A836C
:100F6B00ECFAE0A3C8C582C8CCC583CCF0A3C8C536
:100F7B0082C8CCC583CCDFEADEE880DB89828A833A
:100F8B00E493A3F208DFF980CC88F0EF60010E4EFA
:100F9B0060C388F0ED2402B4040050B9F582EB2451
:100FAB0002B4040050AF2323458223900F1473BB6C
:100FBB00010689828A83E0225002E722BBFE02E30C
:100FCB002289828A83E49322BB010CE58229F58274
:100FDB00E5833AF583E0225006E92582F8E622BB49
:100FEB00FE06E92582F8E222E58229F582E5833ABD
:100FFB00F583E49322BB010689828A83F022500297
:10100B00F722BBFE01F322F8BB010DE58229F58225
:10101B00E5833AF583E8F0225006E92582C8F622EB
:10102B00BBFE05E92582C8F222C5F0F8A3E028F043
:10103B00C5F0F8E582158270021583E038F022A323
:10104B00F8E0C5F025F0F0E582158270021583E01B
:10105B00C838F0E8228A838982E473E56C2582F52F
:10106B0082E56B3583F583B56B0485826C2210AFFB
:10107B000685826CF56B2285826CF56BD2AF22E50F
:10108B006C2582F582E56B3583F5832290FFFB128D
:10109B001066856B83856C82E4F0A3F0856B83858A
:1010AB006C82A3A3F090000312108AE4F09000046A
:1010BB0012108AE4F0856B83856C82F0856B8385D7
:1010CB006C82E0FFC394084003021173EF25E02408
:1010DB00C7F582E43402F58374FFF5F01210344542
:1010EB00F07079856B83856C82E0FF25E0245BF5DE
:1010FB0082E43429F583E493FC740193FDEF25E03E
:10110B0024C7F582E43402F583ECF0A3EDF0856B94
:10111B0083856C82E090296B93856B83856C82A3AE
:10112B00F0856B83856C82A3E0FF9002D7E05F6054
:10113B00059002C58014856B83856C82A3E0FF90BC
:10114B0002D8E0FE5F60089002C6E04FF0800D858C
:10115B006B83856C82A3E04E9002D8F0856B838500
:10116B006C82E004F00210C7C2AF9002D880769078
:10117B00000312108AE0FF856B83856C82A3A3E0CA
:10118B00FEC39F4003021214EE14FF9000041210D2
:10119B008AEFF0C2AF9002D8E0FF90000412108AE1
:1011AB00E0FE90296B93FDF45F9002D8F09002D78C
:1011BB00E04DF0D2AFEE75F003A42492F582E43447
:1011CB0002F583A3E0FAA3E0F9121060C2AF90021C
:1011DB00D7E0FF90000412108AE090296B93F45F24
:1011EB009002D7F0A3E090297393856B83856C8273
:1011FB00A3A3F09002D7E090297393FF9000031202
:10120B00108AEFF0D2AF02117A90000502106690AF
:10121B000309EFF0E4A3F0900286E0FF900117E0E2
:10122B006F606FE490010EF0900004F090010DF0F0
:10123B00900000F0900117EFF090030A7401F0900A
:10124B00030AE0FFC394085049EF902A7393FF9071
:10125B000117E05F90030A701CE0FEEFF45226EEDC
:10126B0075F014A4240EF9740035F0FA7B017D148B
:10127B001224BE8015E0FF902ABB9390010DF090D5
:10128B000000EFF090010EE004F090030AE004F090
:10129B0080AD90010EE0FED394014066E490000314
:1012AB00F0900309E0A3F090030AE0FFC394085009
:1012BB002F900309E0600DEF902A7393FF900117B5
:1012CB00E05F601490030AE0FF902ABB9390000349
:1012DB00F0900309EFF0800890030AE004F080C758
:1012EB00900003E06007900309E0B4080F902AC355
:1012FB00E493900003F09003097408F0900309E065
:10130B00FF22EE6401702D900004E004F0E0FEB4C7
:10131B000102802BEEB40202802E900004E0B40395
:10132B000E90010DE0900003F0900000E0FF229082
:10133B002ABC8034900004E004F0E0FEB401059078
:10134B002AC3801AEEB4020C902ABBE493900003DC
:10135B00F07F0022900004E0B4030A902ABCE493CF
:10136B00900003800B902ABDE493900003F0E4A35C
:10137B00F07F08229002B1E0FF14603924FD605C1D
:10138B001470030214321470030214591460712484
:10139B0007600302147B122407C002C00178B37CE0
:1013AB00027D01D001D0027E007F02120F949002C9
:1013BB00B17401F0229002B1E0FF122407C002C009
:1013CB000178B57C027D01D001D0027E007F021234
:1013DB000F941225979002B17404F0229002B1E0A1
:1013EB00FF122407C002C00178B87C027D01D00136
:1013FB00D0027E007F02120F949002B17407F0228C
:10140B009002B1E0FF122407C002C00178BE7C023B
:10141B007D01D001D0027E007F02120F941225B8FD
:10142B009002B17405F0229002B1E0FF122407C0C4
:10143B0002C00178BA7C027D01D001D0027E007F10
:10144B0002120F941223109002B17406F022900234
:10145B00B1E0FF122407C002C00178BC7C027D0101
:10146B00D001D0027E007F02120F9412234F800016
:10147B00E49002B1F022E4F529A2229248A2239231
:10148B0049A211924AA214924BA212924CA213920D
:10149B004DA221924EA224924F900203E529F0E433
:1014AB00A3F0F529A20C9248A20D9249A20E924AE2
:1014BB00A20F924BA20A924CA20B924DA209924EF2
:1014CB00A208924FA3E529F0E4F529A21A9248A2AB
:1014DB0019B39249A22A924AA229B3924BA21F9204
:1014EB004CA21C924DA22F924EA22C924FA3E529F7
:1014FB00F0E52D24FF9267E433A3F0E4F529A2284D
:10150B0082209248A21882109249A21E924AA22DC2
:10151B008225924BA21D8215924CA22E924DE5E88C
:10152B00F4F528A241924EA227924FA3E529F0C3CE
:10153B00203001D39264E526F4F529900286E0F57C
:10154B0028D240E5295528900209F0A2009263E5C4
:10155B002C549F90020CF0E4A3F022E49002FDF0D7
:10156B00A3F0A3F0A3F090025EE09002FD30E71130
:10157B007403F0A37429F0A37403F0A37415F08023
:10158B000E7402F0A3747BF0A37402F0A3E4F0E4F6
:10159B00F5299002B8E0FCA3E0FDC3900300E09DA9
:1015AB009002FFE09C50179002FDE0FCA3E0FDC30E
:1015BB009002B9E09D9002B8E09C5002D248900294
:1015CB00BEE0FCA3E0FDC3900300E09D9002FFE0B2
:1015DB009C50179002FDE0FCA3E0FDC39002BFE01E
:1015EB009D9002BEE09C5002D249EF75F013A424EB
:1015FB00BEF582E43400F583E054E3F0E5295403AF
:10160B00FEBE0313EF75F013A424BEF582E4340081
:10161B00F583E0441CF022EE7013EF75F013A42455
:10162B00BEF582E43400F583E04408F022EF75F058
:10163B0013A424BEF582E43400F583E04414F022B5
:10164B00E4F529900070E0F528A240926C9000849C
:10165B00E0F528A240926D900082E0FF90006EE0D2
:10166B004FF528A2409249A2419248A242924AC207
:10167B004B900098E0F528A240926E9000ACE0F5FC
:10168B0028A240926F9000AAE0FF900096E04FF5E1
:10169B0028A240924DA241924CA242924EC24F9030
:1016AB00020BE529F0E4F529900020E0FFF528A2D4
:1016BB00409268900034E0F528A240926990003285
:1016CB00E0FE90001EE04EF528A2409249A2419206
:1016DB0048A242924AC24B900048E0F528A24092A1
:1016EB006A90005CE0F528A240926B90005AE0FEF5
:1016FB00900046E04EF528A240924DA241924CA29A
:10170B0042924EC24F90020AE529F0EF5430FF90FF
:10171B000200E04F90020EF0229001E9E0FBA3E003
:10172B00FAA3E0F9120FBA900002F064DD706F902B
:10173B00000A120FD3644F702790000B120FD3B413
:10174B00501E90000C120FD3B44215C25DE9240A4F
:10175B00F9E43AFA780F7C017D017E007F08801E48
:10176B00C251D2549001E9E0FBA3E0FAA3E02402BA
:10177B00F9E43AFA780E7C007D017E007F14120F9B
:10178B0094305D0E900118E004F0E0C394324002F7
:10179B00C25DE4900005F0902A73934226229000DC
:1017AB0002E0FF74DDC39F5047EF94E4504274286E
:1017BB002FF582E434FFF583E4F0EF902996934202
:1017CB00269001E9E0FBA3E0FAA3E02402F9E43A56
:1017DB00FAC001900002E075F014A424CAF974EE6B
:1017EB0035F0A801FC7D01D0017E007F14120F940F
:1017FB0022065E00000000000020302E00000000DA
:10180B0000000000000000000000000000000000CD
:10181B0000000000000000000000000000000000BD
:10182B000000000000000000000000000165FF0147
:10183B0064FF0167FF0166FF4101FF004601E10004
:10184B0000010119004601ED000001017000460185
:10185B00E70000010158004601F300000101CA0036
:10186B004101FCFF4101F9FF4101FEFF4101FDFF79
:10187B00580292FF273EFF005EFF0022FF00F6FF9B
:10188B00266FFF274CFF2758FF228C4102C20041D5
:10189B0002C3004102C4004102AE324102B000411A
:1018AB0002B1004102C1004102B2004102B7000087
:1018BB00E490030EF0900285E09002B0F090028469
:1018CB00E030E07720593D30583AC2589002C3E0DF
:1018DB00FF9002C2F09002C4E09002C3F09002B0FD
:1018EB00E09002C4F0B5071C9002C3E0FF9002B079
:1018FB00E0FEB5070F9002C4E0FFEEB507069003BC
:10190B000EF0D25930593B205B387F007EE0122518
:10191B00D97B017A03790E7F007EE01225547B017F
:10192B007A0279AF7F007EE012253290030EE0FF42
:10193B009002AFE0B5070BD25B8007C259C25B12B6
:10194B002576E4F529A25A924BA25B924A900200AB
:10195B00E529F022787FE4F6D8FD9000007F007E29
:10196B0004E4F0A3DFFCDEFA756B04756C00758183
:10197B006C0219BA021DCAE493A3F8E493A34003C3
:10198B00F68001F208DFF48029E493A3F8540724CE
:10199B000CC8C333C4540F4420C8834004F456808E
:1019AB000146F6DFE4800B01020408102040809012
:1019BB0017FCE47E019360BCA3FF543F30E5095450
:1019CB001FFEE493A360010ECF54C025E060A84036
:1019DB00B8E493A3FAE493A3F8E493A3C8C582C82D
:1019EB00CAC583CAF0A3C8C582C8CAC583CADFE902
:1019FB00DEE780BE900291E0B48103D38001C392F5
:101A0B005C90025FE0FFF529A24892A4A24992A341
:101A1B00A24B92A2A3E0FEF529A24892A7A249925B
:101A2B00A6A24B92A590025CE0FDF529A24AB392C7
:101A3B00A08E29A24FB392A1A3E0F529A24E923F0B
:101A4B008D29A24B923AA24C923B900020E0F528B4
:101A5B00305009A253B39238D23980282051033029
:101A6B00520AA2569238A257923980182048033056
:101A7B004103D38001C39238204903304203D38002
:101A8B0001C39239A2389256A23992578F29A24C90
:101A9B00923C229001F4E024FEFF9001F3E0C39FFF
:101AAB00504E9001F5E0FBA3E0FAA3E0F99001F3AF
:101ABB00E0FFF582758300120FD3FE9001FEE06EFE
:101ACB009001FBF0E090275B93FD9001FDE0FCEDB6
:101ADB006CA3F09001FBE090285B939001FDF0EE7E
:101AEB00A2D0929B8F82758300120FD3F59980320F
:101AFB009001F4E0FF24FEFE9001F3E0FDB5060536
:101B0B009001FE8008EF14B5050C9001FDE0A2D00A
:101B1B00929BF599800CD2E89001FE74FFF0900136
:101B2B00FDF09001F3E004F0229001EEE024FEFFC3
:101B3B009001EDE0FDC39F503C9001EFE0FBA3E073
:101B4B00FAA3E0F98D82758300120FD3FE656790BF
:101B5B0001FAF0E0FF90275B936566F567EF90283D
:101B6B005B93F566EEA2D0929B8D82758300120F6C
:101B7B00D3F599802B9001EEE0FF24FEFE9001ED52
:101B8B00E0FDB50604E5678007EF14B5050AE566C9
:101B9B00A2D0929BF5998008D2B37567FF7566FF4B
:101BAB009001EDE004F02290030CEFF0700A305D31
:101BBB00079000BEE04480F090030CE0FF2405F595
:101BCB0082E43400F583E0FE6008EF902A7393F40F
:101BDB005226EE6414703290030CE07008D251C29E
:101BEB00659001FFF090030CE0FF2405F582E434CF
:101BFB0000F583E4F0EF75F014A4240EF9740035AE
:101C0B00F0FA7B017D141224BE90030CE02405F541
:101C1B0082E43400F583E004F022E4F52990001F00
:101C2B00E0FFF528A2429248A240B39249A2439208
:101C3B004B90006FE0FEEF4EF528A241924AA2476F
:101C4B00924CA21B924DA22B924EA216B3924F9086
:101C5B000201E529F0E4F52990001EE0F528A243E6
:101C6B009249A244924AA245924BA246924CA24759
:101C7B00924EA3E0F528A2449248A246924DA2456B
:101C8B00924F900202E529F022900003E0FE9001B2
:101C9B00F5E0FBA3E0FAA3E0F9EE1210009001F5DA
:101CAB00E0FBA3E0FAA3E0F99000017465121012B7
:101CBB00EF75F013A424AEF9740035F0FA7B01C074
:101CCB0003C002C0019001F5E0FBA3E0FAA3E024FE
:101CDB0002F9E43AA801FCAD03D001D002D0037E97
:101CEB00007F13120F941226D8C2E8AEAC75AC016C
:101CFB00D299AF068FAC229001ECE0705E9001E7B9
:101D0B00E0FFC3941850549001E9E0FBA3E0FAA361
:101D1B00E0F98F82758300E5991210128F8275831B
:101D2B0000120FD3FF9001FCE06F9001FBF0E0FC81
:101D3B0090275B93FE9001F9E0FDEE6D9001FCF0B6
:101D4B00EC90285B939001F9F09001E7E004F090A0
:101D5B0002F7E0F58DA3E0F58BD28E22E490030B16
:101D6B00F0F090030BE0FFC3940650111226FF9086
:101D7B00030BE0245EF8A607E004F080E5635EFF4A
:101D8B00E490030BF090030BE0FFC39406502FEF8E
:101D9B0075F008A4242EF9E4FAFBC001E0FE245EE2
:101DAB00F8E6FF74202EF9E49002E6F0A3F0A3E925
:101DBB00F0D00112006690030BE004F080C722E420
:101DCB00FFFE1221731226591226EC7B017A02793F
:101DDB00AF7F007EE012253212272112002612243B
:101DEB00E812262912264112250D12243A12001E42
:101DFB001200031224667DFF7F071225F6E4FEFF17
:101E0B000FBF00010EBEFFF8BFFFF5E4FD7F071209
:101E1B0025F6D25ED250D25DD2AF12005680FBC0F7
:101E2B00E0C0F0C083C082C0D075D000C000C0013C
:101E3B00C002C003C004C005C006C007900305E480
:101E4B00F0E5ACF075AC00309807C298121F3A80E1
:101E5B0008309905C299121B34900305E0F5ACD0FC
:101E6B0007D006D005D004D003D002D001D000D0CB
:101E7B00D0D082D083D0F0D0E032C0E0C0F0C083AD
:101E8B00C082C0D075D000C000C001C002C003C06A
:101E9B0004C005C006C007900306E4F0E5ACF0757E
:101EAB00AC01309807C298121D028008309905C208
:101EBB0099121A9E900306E0F5ACD007D006D00518
:101ECB00D004D003D002D001D000D0D0D082D083A8
:101EDB00D0F0D0E032C0E0C0F0C083C082C0D0757B
:101EEB00D000C000C001C002C003C004C005C006C2
:101EFB00C0077BFF7A00790A8B688A69896AC2AF4F
:101F0B0075D80075F9A275E94075D840121060D2EA
:101F1B00AF121097D007D006D005D004D003D00253
:101F2B00D001D000D0D0D082D083D0F0D0E032908E
:101F3B0001E6E070509001E1E0FFC3943F50469002
:101F4B0001E3E0FBA3E0FAA3E0F98F82758300E5E0
:101F5B00991210128F82758300120FD36565900151
:101F6B00FAF0E0FF90275B936564F565EF90285BD3
:101F7B0093F5649001E1E004F09002F5E0F58CA399
:101F8B00E0F58AD28C229001E3E0FBA3E0FAA3E018
:101F9B00F9120FBA64D27042900001120FD364652C
:101FAB007038E5657034E56470309002C0F09002D3
:101FBB00AAF0C25FD258D255C25212203A9001E316
:101FCB00E0FBA3E0FAA3E02402F9E43AFA78577CA9
:101FDB00027D017E007F3B120F94229001E9E0FB12
:101FEB00A3E0FAA3E0F9120FBAFF900003E06F70C1
:101FFB003D900001120FD3646570339001FCE070CB
:10200B002D9001F9E070279001E7E0FFB418112043
:10201B0065199001FFE004F0E0B4030FD265800B6B
:10202B00EFB41707C265E49001FFF012172422905A
:10203B0001EFE0FBA3E0FAA3E0F974D212100090D9
:10204B0001EFE0FBA3E0FAA3E0F990000174651245
:10205B0010129001EFE0FBA3E0FAA3E02402F9E4F5
:10206B003AA801FCAD037B017A0279017E007F5611
:10207B00120F94C2B3122711AFACE4F5ACD2998F07
:10208B00AC229002D9EBF0A3EAF0A3E9F0E4FF7ED7
:10209B00079002DFE0FBA3E0FAA3E0F98E827583E1
:1020AB0000120FD3FD9002DCE0FBA3E0FAA3E0F9F2
:1020BB008E82758300120FD34DFD9002D9E0FBA3E6
:1020CB00E0FAA3E0F98F82758300ED1210121E0F58
:1020DB00EFB408BD22900001E0D394085003305DAB
:1020EB0005E4900001F0900001E0FF12121A90003D
:1020FB0001EFF0E0FF902ABB93FE900003E0B506E2
:10210B0017121BB2900001E0C313FF120C88900052
:10211B0001E0C313FF121C94900001E004F0222095
:10212B005F269002C0E0D394144016E4F0D2527BA9
:10213B00017A0279577D3B1224BE7565FF7564FFEA
:10214B00229002C0E004F0227B017A0279577D3B9A
:10215B001224BEE4900257F0A37452F0E490028173
:10216B00F0A3F0A374FAF022E4900304F0C28C43C2
:10217B008901758CDCF58AC28D122685900304EFDC
:10218B00F04408FFF012269AD28C308DFDC28DC21E
:10219B008C122685900304EFF04403FFF012269A6D
:1021AB00122685900304EFF054FBFFF002269AC031
:1021BB00E0C0F0C083C082C0D075D000C000C001A9
:1021CB00C002C003C004C005C006C007C28C90018A
:1021DB00E67401F0121F911226AFD007D006D0057E
:1021EB00D004D003D002D001D000D0D0D082D08385
:1021FB00D0F0D0E032C0E0C0F0C083C082C0D07558
:10220B00D000C000C001C002C003C004C005C0069E
:10221B00C007C28E9001EC7401F0121FE61226105B
:10222B00D007D006D005D004D003D002D001D00007
:10223B00D0D0D082D083D0F0D0E0329002F9EBF046
:10224B00A3EAF0A3E9F0E4A3F0FF9002F9E0FBA30B
:10225B00E0FAA3E0F98F82758300120FD3FEEED361
:10226B00940040159002FCE004F0E0D3940140038D
:10227B007F0122EE145EFE80E50FEFB408CC7F00E9
:10228B0022205F0E9002AAE004F0E0C39408400203
:10229B00D25F305E2D9002ACE004F070069002AB82
:1022AB00E004F09002ABE07004A3E0640A701390BA
:1022BB0002ABF0A3F0C25E30500820510330520243
:1022CB00D253229002EFEBF0A3EAF0A3E9F0E4FF84
:1022DB007E07EFC39408502C9002F2E0FBA3E0FAC8
:1022EB00A3E0F98E82758300120FD3FD9002EFE00D
:1022FB00FBA3E0FAA3E0F98F82758300ED121012B5
:10230B000F1E80CE22C39002BBE094849002BAE0F1
:10231B009400501DA3E0941E9002BAE0940140116A
:10232B009002B2E0B43205D26214F0229002B28075
:10233B00089002B2E07006C262E004F0229002B292
:10234B00E014F022C39002BDE094219002BCE09413
:10235B0001501DA3E094849002BCE09402401190C4
:10236B0002B7E0B43205D26114F0229002B78008B4
:10237B009002B7E07006C261E004F0229002B7E071
:10238B0014F0229002E9EBF0A3EAF0A3E9F0E4FFEA
:10239B007E079002ECE0FBA3E0FAA3E0F98E8275D6
:1023AB008300120FD3FD9002E9E0FBA3E0FAA3E058
:1023BB00F98F82758300ED1210121E0FEFB408D245
:1023CB002290020174AAF0A37455F078037C027D6D
:1023DB00017BFF7A2A79D47E007F08120F94780B49
:1023EB007C027D017B017A01790F7E007F08120F41
:1023FB009490021374AAF0A37455F02253C5F8EF0E
:10240B0042C543C588E5C530E4FB53C5EFE5C6259A
:10241B00E025E0FFE5BE54034F900308F0E5C6C48A
:10242B0013135403900307F07B017A03790722E41B
:10243B00FFEF25E0245BF582E43429F583E493FC7C
:10244B00740193FDEF25E024C7F582E43402F58394
:10245B00ECF0A3EDF00FEFB408D722E4FFEF75F02B
:10246B0013A424BFF582E43400F583E04440F0EF7D
:10247B0075F013A424BFF582E43400F583E030E655
:10248B00EE0FEFB408D7227F081226FFBFFF119083
:10249B0002ADE07004C26080169002ADE014F02231
:1024AB009002ADE0B40A05D26014F0229002ADE0C8
:1024BB0004F022900301EBF0A3EAF0A3E9F0E4FFB0
:1024CB00EFC39D5017900301E0FBA3E475F00112DD
:1024DB00104AA9F0FAE41210000F80E42275AC0147
:1024EB007598D0759AFAE4F5AC9002F774FDF0A3E9
:1024FB0074F0F0439A1443AE1043AF1043AD10D2B7
:10250B00E82275D903E4F5DAF5DBF5DCF5DDF5DE6C
:10251B00F5DFF5D875F9A275E94053AEFB53AFFB68
:10252B0075D84043AD0422AD07AC0675E78175E560
:10253B0001ECF5E3EDF5E4AFA8C2AF75E64675E641
:10254B00B9E5E21210008FA822AD07AC0675E78142
:10255B0075E502ECF5E3EDF5E4120FBAF5E2AFA881
:10256B00C2AF75E64675E6B98FA8229002B0E0FFC0
:10257B009002AFE0B50709D25A9002AE7432F02246
:10258B009002AEE014F0E07002C25A229002B3E067
:10259B0090022FF09002B4E0900230F09002B5E080
:1025AB00900231F09002B6E0900232F0229002B825
:1025BB00E0900233F09002B9E0900234F09002BE4A
:1025CB00E0900235F09002BFE0900236F022AD07AA
:1025DB00AC06ECF5E3EDF5E475E50375E781AFA823
:1025EB00C2AF75E64675E6B98FA822900304EDF0ED
:1025FB001226C4900304E0F580E4FF0FEFB41EFB3A
:10260B00D2B7D2B722E49001E7F0A37418F0E490AC
:10261B0001ECF09001FC74FFF09001F9F02253A64D
:10262B007F4389019002F5E0F58CA3E0F58A43B86E
:10263B0002D2A9C28C2253A6BF4389109002F7E0A5
:10264B00F58DA3E0F58B43B808D2ABC28E22E4FF25
:10265B0075AD08122685EF4440FF12269A43AF084A
:10266B0043AE0822122730205C081219FF122752A2
:10267B0080051223CCC25C02212AE4F5E375E50741
:10268B0043E78075E64675E6B953E77FAFE2228FE5
:10269B00E275E50643E78075E64675E6B9E4F5E5D0
:1026AB0053E77F22E49001E1F0A3743FF0E4900143
:1026BB00E6F07565FF7564FF22EFC39408500A536B
:1026CB00B00FEFC454F042B02243B08022E490012B
:1026DB00F3F0A37417F09001FE74FFF09001FDF07E
:1026EB002275E2E075E50475E78175E64675E6B996
:1026FB0075E701221226C47580FFE4FF0FEFB40AC1
:10270B00FBAF80D2B722E49001EDF0A3745AF075C1
:10271B0067FF7566FF227591F3E4F592F595759653
:10272B00FF43A00322AD277F061225F6AD267F07B8
:10273B000225F6121D67305407305504C250C253A0
:10274B00221218BB02249212000E021481B2EA224A
:10275B0000C1814001C0804101C0804100C1814066
:10276B0001C0804100C1814000C1814001C0804156
:10277B0001C0804100C1814000C1814001C0804146
:10278B0000C1814001C0804101C0804100C1814036
:10279B0001C0804100C1814000C1814001C0804126
:1027AB0000C1814001C0804101C0804100C1814016
:1027BB0000C1814001C0804101C0804100C1814006
:1027CB0001C0804100C1814000C1814001C08041F6
:1027DB0001C0804100C1814000C1814001C08041E6
:1027EB0000C1814001C0804101C0804100C18140D6
:1027FB0000C1814001C0804101C0804100C18140C6
:10280B0001C0804100C1814000C1814001C08041B5
:10281B0000C1814001C0804101C0804100C18140A5
:10282B0001C0804100C1814000C1814001C0804195
:10283B0001C0804100C1814000C1814001C0804185
:10284B0000C1814001C0804101C0804100C1814075
:10285B0000C0C101C30302C2C60607C705C5C40435
:10286B00CC0C0DCD0FCFCE0E0ACACB0BC90908C8A5
:10287B00D81819D91BDBDA1A1EDEDF1FDD1D1CDC95
:10288B0014D4D515D71716D6D21213D311D1D01005
:10289B00F03031F133F3F23236F6F737F53534F4F5
:1028AB003CFCFD3DFF3F3EFEFA3A3BFB39F9F83865
:1028BB0028E8E929EB2B2AEAEE2E2FEF2DEDEC2C55
:1028CB00E42425E527E7E62622E2E323E12120E0C5
:1028DB00A06061A163A3A26266A6A767A56564A4B5
:1028EB006CACAD6DAF6F6EAEAA6A6BAB69A9A86825
:1028FB0078B8B979BB7B7ABABE7E7FBF7DBDBC7C15
:10290B00B47475B577B7B67672B2B373B17170B084
:10291B005090915193535292965657975595945474
:10292B009C5C5D9D5F9F9E5E5A9A9B5B99595898E4
:10293B00884849894B8B8A4A4E8E8F4F8D4D4C8CD4
:10294B004484854587474686824243834181804044
:10295B00000100040005000A0014003200FA01F423
:10296B000102040810204080090102010301020149
:10297B00040102010301020105010201030102012D
:10298B00040102010301020106010201030102011C
:10299B00040102010301020105010201030102010D
:1029AB0004010201030102010701020103010201FB
:1029BB0004010201030102010501020103010201ED
:1029CB0004010201030102010601020103010201DC
:1029DB0004010201030102010501020103010201CD
:1029EB0004010201030102010801020103010201BA
:1029FB0004010201030102010501020103010201AD
:102A0B00040102010301020106010201030102019B
:102A1B00040102010301020105010201030102018C
:102A2B00040102010301020107010201030102017A
:102A3B00040102010301020105010201030102016C
:102A4B00040102010301020106010201030102015B
:102A5B00040102010301020105010201030102014C
:102A6B00040102010301020101020408102040804D
:102A7B0000000201030704080509060A0700090004
:102A8B000A000C0B0D000B00080F0F0000030000D9
:102A9B00000000000201030704080509060A0700ED
:102AAB00080F090D0A000B000C0B0D000E000F0098
:102ABB00DDDEDFE0E1E2E3E4DCFEFDFBF7EFDFBFB1
:102ACB007F01020408102040805344434146325298
:012ADB0036C4
:00000001FF
